:020000040800F2
:1000000000040220010200084D0F0008510F0008F3
:10001000A50F0008510F0008790F0008030200081F
:100020000302000803020008030200087128000808
:10003000030200080302000803020008030200088C
:10004000030200080302000803020008030200087C
:100050000302000803020008893A0008B53A0008C4
:10006000E13A00080D3B0008393B00080302000894
:10007000030200080302000803020008030200084C
:10008000030200080302000803020008030200083C
:10009000030200080302000803020008653B000891
:1000A000030200080302000803020008030200081C
:1000B000AD3800080302000803020008030200082C
:1000C00003020008030200080302000803020008FC
:1000D0000302000803020008591100086D1100080E
:1000E000CD3B0008030200080302000803020008D9
:1000F00003020008030200080302000803020008CC
:1001000003020008030200080302000803020008BB
:1001100003020008030200080302000803020008AB
:10012000030200080302000803020008030200089B
:10013000030200080302000803020008030200088B
:10014000030200080302000803020008DD2F000874
:10015000030200080302000803020008030200086B
:10016000030200080302000803020008030200085B
:10017000030200080302000803020008030200084B
:1001800003020008030200088111000803020008AE
:10019000030200080302000803020008030200082B
:1001A000030200080302000803020008030200081B
:1001B000030200080302000803020008030200080B
:1001C00003020008030200080302000803020008FB
:1001D00003020008030200080302000803020008EB
:1001E00003020008030200080302000803020008DB
:1001F00003020008030200080302000803020008CB
:1002000002E000F000F8FEE772B6394880F3088893
:10021000384880F3098838484EF60851CEF200017C
:10022000086040F20000CCF200004EF63471CEF2CD
:1002300000010860BFF34F8FBFF36F8F40F20000E3
:10024000C0F2F0004EF68851CEF200010860BFF314
:100250004F8FBFF36F8F4FF00000E1EE100A4EF6A4
:100260003C71CEF200010860062080F31488BFF3D1
:100270006F8F02F03BFB03F0A1FA4FF055301F499E
:100280001B4A91423CBF41F8040BFAE71C49194A4A
:1002900091423CBF41F8040BFAE71A491A4A1B4B3A
:1002A0009A423EBF51F8040B42F8040BF8E70020D5
:1002B0001749184A91423CBF41F8040BFAE702F093
:1002C00059FB03F0E5FA144C144DAC4203DA54F830
:1002D000041B8847F9E700F03FF8114C114DAC4280
:1002E00003DA54F8041B8847F9E702F041BB000029
:1002F0000004022000240220000000080000022068
:10030000000402204840000800240220502402205B
:1003100050240220B03D0220000200080002000824
:1003200000020008000200082DE9F04F2DED108AB0
:10033000C1F80CD0D0F80CD0BDEC108ABDE8F08F1D
:10034000002383F311882846A047002001F016FF00
:1003500001F0C6FE00DFFEE770B5204C78230025D3
:1003600023706FF07F061E236570A570E570257100
:100370006571A571E57125726672A372E57200F070
:100380002DFD20B10E2325726672A372E57202F074
:1003900031FA044602F066FA0546D8B9104B9C4281
:1003A0001AD001339C4218BF054641F2883404BF7D
:1003B00001250024002002F027FA0DB100F0B6F864
:1003C00000F066FD00F05CFC204600F04FF900F004
:1003D000ADF8F9E70024EDE70446EBE750240220EE
:1003E000010007B008B500F0C9FBA0F12003584296
:1003F000584108BD07B5054B02211B88ADF80430F4
:1004000001A800F027FC03B05DF804FBB43C000831
:10041000064991F8243033B100230822086A81F894
:10042000243000F051BC0120704700BF702402202E
:100430002DE9F84F234C94F824300546884617469A
:100440008BBB2E46DFF87C90002F38D094F824A088
:10045000BAF1000F05D12022FF214846266200F0A4
:1004600005FDCAF10805BD4228BF3D465FFA85FB80
:10047000AD0041462A4604EB8A0000F0CDFC94F81A
:100480002430A7EB0B079B445FFA8BFBBBF1080FF3
:100490002E44A844FFB284F824B0D5D1FFF7B8FFAA
:1004A0000028D1D108E0266A06EB8306B042C9D005
:1004B000FFF7AEFF0028C4D10020BDE8F88F01206F
:1004C000BDE8F88F7024022010B5202383F3118833
:1004D0001248C3680BB101F0D7FE0023104A0F4841
:1004E0004FF47A7101F094FE002383F311880D4CD0
:1004F000236813B12368013B2360636813B1636809
:10050000013B6360084B1B7833B9636823B9022051
:1005100000F080FC3223636010BD00BF5C24022029
:10052000C9040008A0250220982402202DE9F041EA
:10053000444B454953F8042F013201D1BDE8F08105
:100540008B42F7D1414C424B22689A4278D9414BB9
:100550009B6803F1006303F5C0339A4270D2002018
:1005600000F0AAFB3C4B0220187000F051FC3B4B02
:100570001A6C00221A64196E1A66196E596C5A6444
:10058000596E5A66596E596941F08001596159692D
:1005900021F0800159615969196941F000511961CF
:1005A000196921F0005119611B6972B62C492D4B54
:1005B0000B601D682468BFF34F8FBFF36F8F2A4B0A
:1005C000C3F88420BFF34F8F5A6922F480325A61F6
:1005D000BFF34F8FD3F88020C2F3C906C2F34E3267
:1005E0005201B70743F6E07E02EA0E08384631466C
:1005F000013948EA000CB1F1FF3FC3F874C200F1C1
:100600004040F5D1203A12F1200FEDD1BFF34F8FCA
:10061000BFF36F8FBFF34F8FBFF36F8F5A6922F411
:1006200000325A610022C3F85022BFF34F8FBFF34C
:100630006F8F202383F31188AD4685F30888204708
:10064000BDE8F081FC7F01081C80010804800108DE
:10065000FF7F010850240220982402200038024025
:1006600008ED00E00080010800ED00E02DE9F04F0A
:1006700099B0B34C01902022FF2110A8A66800F089
:10068000F5FBB04A1378A346A3B9AF480121C36074
:100690001170202383F31188C3680BB101F0F4FDBE
:1006A0000023AA4AA8484FF47A7101F0B1FD002353
:1006B00083F31188019B13B1A54B019A1A60A54AD7
:1006C000A349019F0292002313704B6099461C4678
:1006D0001D469846012000F09BFB002F00F012827F
:1006E0009B4B1B68002B40F00D8219B0BDE8F08FCA
:1006F0000220FFF777FE002840F0FB81019BB9F153
:10070000000F08BF1F46944B1B88ADF82C30022108
:100710000BA800F09FFADDE74FF47A7000F02EFA94
:10072000031E0393EADB0220FFF75CFE82460028EB
:10073000E4D0039B581E042800F2DD81DFE800F0BE
:10074000030E1114170018A8052340F8343D0421A6
:1007500000F080FA54464FF0000856E00421784833
:10076000F6E704217D48F3E704217D48F0E71C24E7
:10077000204600F0A3FA04340B9004210BA800F0EB
:1007800069FA2C2CF4D1E5E7002DB7D0002CB5D0B8
:100790000220FFF727FE0546002800F0AF81012068
:1007A0006C4C00F089FA0220207000F031FB4FF011
:1007B00000095FFA89FA504600F08EFA074658B1F0
:1007C000504600F099FA09F101090028F1D12C46B0
:1007D000A9460027634B97E701230220237000F00E
:1007E00015FB3E46DBF808309E4206D2304600F04C
:1007F00065FA0130EBD10436F4E7029B00261E7047
:10080000534BA9465E602C46374600F037FB15B1C6
:10081000002C18BF0027FFF7EDFD5BE7002D3FF42C
:100820006DAF002C3FF46AAF029B0220187000F0FD
:10083000EFFA322000F0A2F9B0F1000AC0F25E81B6
:100840001AF0030540F05A81DBF8082006EB0A0392
:10085000934200F25381BAF5807F00F24F815545F3
:100860000DDA4FF47A7000F089F90490049B002BA4
:10087000C0F244813C4A049BAB540135EFE7C820E9
:10088000FFF7B0FD0546002800F038811F2E11D873
:10089000C6F12004544528BF544610AB26F003008F
:1008A00022463149184400F0B7FA2246FF212E486B
:1008B00000F0DCFA4FEAAA0A5FFA8AF22A493046C7
:1008C000FFF7B6FD0446002800F01A8106EB8A0601
:1008D00005469AE70220FFF785FD00283FF40EAF9A
:1008E000FFF796FD00283FF409AF4FF0000A53468A
:1008F000DBF8082092451CD2BAF11F0F12D8109ACB
:1009000001320FD02AF0030218A90A4452F8202C11
:100910000B92184604220BA900F058FB0AF1040AB6
:100920000346E5E75046039300F0C8F9039B0B909C
:10093000EFE718A8042140F84C3D00F08BF964E77C
:10094000502402209C2502205C240220C9040008B7
:10095000A025022098240220B63C0008542402203E
:1009600058240220B83C00089C24022018A8002328
:1009700040F8343D642100F039F900287FF4BEAE20
:100980000220FFF72FFD00283FF4B8AE0B9800F0CF
:10099000C5F918AB43F8480D04211846CDE718A84F
:1009A000002340F8343D642100F020F900287FF452
:1009B000A5AE0220FFF716FD00283FF49FAE0B986E
:1009C00000F0BAF918AB43F8440DE5E70220FFF751
:1009D00009FD00283FF492AE00F0B4F918AB43F8DB
:1009E000400DD9E70220FFF7FDFC00283FF486AE5A
:1009F0000BA9142000F0ACF9824618A8042140F895
:100A00003CAD00F027F951460BA896E7322000F0E4
:100A1000B5F8B0F1000AFFF671AE1AF0030F7FF4DB
:100A20006DAEDBF808200AEB080393423FF666AE92
:100A30000220FFF7D7FC00283FF460AE2AF0030A3B
:100A4000C244D0453FF4E1AE404600F037F90421FE
:100A50000A900AA800F0FEF808F10408F1E74FF444
:100A60007A70FFF7BFFC00283FF448AEFFF7D0FCD8
:100A700000283FF4AFAE109B01330CD0082210A920
:100A80000020FFF7D5FC00283FF4A4AE2022FF2170
:100A900010A800F0EBF9FFF7ADFC374801F074FB4C
:100AA00023E6002D3FF42AAE002C3FF427AE18A811
:100AB000002340F8343D642100F098F88246002875
:100AC0007FF41CAE0220FFF78DFC00283FF416AE29
:100AD0000390FFF78FFC41F2883001F055FB0B9833
:100AE00000F014FA00F0CAF9039B57461C461D4655
:100AF000F0E5054689E64FF00008FFE52546FDE5EF
:100B00002C4667E6002000F039F80490049B002B87
:100B1000FFF6E3AD012000F079F9049B213B122B95
:100B20003FF6D8AD01A252F823F000BFF10600084D
:100B30001907000889070008D5060008D50600082F
:100B4000D50600081D0800080D0A0008D508000891
:100B50006D0900089F090008CD090008D5060008A6
:100B6000E5090008D50600085F0A00080B08000820
:100B7000D5060008A30A0008A08601002DE9F34766
:100B800002AE00244FF47A7506F8014D144FDFF8D9
:100B90005880454397F900305A1C5FFA84F901D018
:100BA000A34212D158F8240003680122D3F820A0F0
:100BB00031462B46D047012807D10A4B9DF8070044
:100BC00083F8009002B0BDE8F0870134042CE1D135
:100BD0004FF4FA7001F0D8FA4FF0FF30F2E700BF9F
:100BE00000240220C4250220C43C00082DE9F0475F
:100BF0004FF47A75144FDFF8588006464D430024B1
:100C000097F900305A1C5FFA84F901D0A34210D141
:100C100058F8240003680422D3F820A031462B465C
:100C2000D047042805D1094B83F800900020BDE887
:100C3000F0870134042CE3D14FF4FA7001F0A4FAE8
:100C40004FF0FF30BDE8F08700240220C4250220C9
:100C5000C43C000830B4074B1A78074B53F82240C5
:100C60002368DD69054B0A46AC460146204630BC88
:100C7000604700BFC4250220C43C0008A0860100D4
:100C8000F8B501F0BBFC094C094E0A4F2070002555
:100C900030682378834207D901F0AAFC3368054401
:100CA0000133BD423360F3D9F8BD00BFC525022032
:100CB000A8250220FF7F010001F04EBD00F1006079
:100CC00000F5C0300068704700F10060920000F548
:100CD000C03001F0D9BC0000054B1A68054B1B78E9
:100CE0009B1A834202D9104401F082BC0020704755
:100CF000A8250220C525022038B5074D04462868DE
:100D0000204401F07DFC28B928682044BDE8384023
:100D100001F08EBC38BD00BFA825022010F00303EF
:100D200008D1B0F5806F05D800F10050A0F5712012
:100D30000068704700207047014BC058704700BFE3
:100D400020F4F01F014B1868704700BF002004E03A
:100D5000F0B5204B1E68204B1F885D6893F9084052
:100D6000C6F30B02BA424FEA164622D09F89BA4216
:100D700021D01F8BBA4206D102220C2404FB02337D
:100D80005D6893F90840B6F5805F16D041F2010323
:100D90009E4208BF5A24421E0A44013D0B4693421C
:100DA00015D215F9016F581C4EB1034600F8016CBD
:100DB000F5E70022E1E70122DFE74124EBE72C25FC
:100DC00082421D7001D9981C5C70401AF0BD184613
:100DD000FBE700BF002004E004240220094B5B88ED
:100DE000B3F5805F09D041F20102934207D101229D
:100DF000054B03EB8203D87870470022F8E7002008
:100E0000704700BF002004E0BC3C000870470000B1
:100E1000704700007047000010B50023934203D0D4
:100E2000CC5CC4540133F9E710BD000030B5441E5A
:100E300014F9010F0B4660B193F90050854201F19E
:100E4000010106D11AB993F90020801A30BD013A88
:100E5000EEE7002AF7D1104630BD000002460346F7
:100E6000981A13F9011B0029FAD17047024403466E
:100E7000934202D003F8011BFAE77047024B1A783D
:100E8000024B1A70704700BFC425022000240220C4
:100E9000F8B5184C1848194D194E174F00F0B4FC0E
:100EA0002146154800F0DCFC24681648E26ED2F8B2
:100EB000043843F00203C2F8043801F065F9204613
:100EC000114900F0DBFDE26ED2F8043823F0020392
:100ED000C2F804384FF4E1332B60002456F82400A4
:100EE000B84202D0294600F0EDFB0134042CF5D1C4
:100EF000F8BD00BFBC3D0008CC330220AC25022069
:100F0000C43C000840420F00E83D000838B50B4BD8
:100F10001A780B4B53F822400A4B9C4205460CD0E2
:100F2000094B002118461822FFF7A0FF0560014673
:100F30002046BDE8384000F0C5BB38BDC4250220BE
:100F4000C43C0008CC330220AC250220FEE70000A0
:100F500000B59BB0EFF3098168226846FFF75CFF9C
:100F6000EFF30583034B9A6B9A6A9A6A9A6A9A6AB4
:100F70009B6AFEE700ED00E000B59BB0EFF309814E
:100F800068226846FFF748FFEFF30583044B9A6B2E
:100F90009A6A9A6A9A6A9A6A9A6A9B6AFEE700BF94
:100FA00000ED00E000B59BB0EFF3098168226846D0
:100FB000FFF732FFEFF30583034B5A6B9A6A9A6A85
:100FC0009A6A9A6A9B6AFEE700ED00E030B5084D28
:100FD0000A4491420BD011F8013B09245840013CCE
:100FE000F7D040F300032B4083EA5000F7E730BD11
:100FF0002083B8ED002304491A465A50C818083314
:10100000802B4260F9D17047C825022002684368EE
:101010001143016003B1184770470000024A13688A
:1010200043F0C0031360704700440040024A136855
:1010300043F0C0031360704700480040024A136841
:1010400043F0C00313607047007800402DE9F0477B
:10105000C66D3768F46934620546200719D014F06C
:10106000080F0CBF00218021E20748BF41F020019A
:10107000A30748BF41F04001600748BF41F48071B9
:10108000202383F31188281DFFF7C0FF002383F37B
:101090001188E2050AD5202383F311884FF40071EB
:1010A000281DFFF7B3FF002383F311884FF02009B9
:1010B0004FF0000A14F0200831D13B0616D54FF04E
:1010C000200905F1380A200610D589F31188504609
:1010D00000F06CFA00282FDA0821281DFFF796FF90
:1010E00027F080033360002383F3118879060DD540
:1010F00062060BD5202383F31188EA6C2B6D9A428C
:1011000001D12B6CEBB9002383F31188E30620D5C2
:10111000AA6E1369EBB15069BDE8F047184789F32F
:101120001188736A95F864102846194000F0D8FABF
:101130008AF31188F469BDE7B06288F31188F46915
:10114000C1E71021281D27F04007FFF75FFF376038
:10115000D9E7BDE8F087000008B50348FFF776FF40
:10116000BDE8084001F094BB4826022008B50348BA
:10117000FFF76CFFBDE8084001F08ABBB4260220EF
:1011800008B50348FFF762FFBDE8084001F080BBE7
:101190002027022037B52D4C2D4D204600F086FA31
:1011A000009404F1140000234FF40072294900F068
:1011B00047F94FF40072009404F13800264B274998
:1011C00000F0C0F9264BE3652566264C0B2126204E
:1011D00000F0C4F8204600F069FA009404F114000D
:1011E00000234FF40072204900F02AF94FF40072F6
:1011F000009404F138001D4B1D4900F0A3F91D4B6C
:10120000E36525661C4C0B21272000F0A7F820463B
:1012100000F04CFA04F11400009400234FF4007223
:10122000164900F00DF904F138000094144B1549EB
:101230004FF4007200F086F9134BE3650B21522046
:10124000256603B0BDE8304000F088B8482602208B
:1012500080F937038C2702201D1000088C2D0220F6
:1012600000440040B42602208C2902202D100008E2
:101270008C2F022000480040202702208C2B0220C7
:101280003D1000088C310220007800402E4B0029D0
:1012900008BF1946037C8166012B30B50CD12B4B5E
:1012A000984235D12A4B1A6C42F400321A641A6EF5
:1012B00042F400321A661B6E0A68036EC46D03EBBB
:1012C0005203B3FBF2F34A68150442BF23F007054B
:1012D00003F0070343EA4503E3608B6843F04003F0
:1012E0006360CB6843F00103A36042F4967343F05C
:1012F0000103236051054FF0FF33236205D512F03F
:1013000010221DD0B2F1805F1CD080F8643030BD57
:10131000104B984208D10E4B1A6C42F480221A648A
:101320001A6E42F48022C5E70B4B9842C4D1084B99
:101330001A6C42F080421A641A6E42F08042B9E799
:101340007F23E2E73F23E0E7003D00084826022034
:1013500000380240B42602202027022000F160431A
:1013600000F01F02400903F5614309018000C9B282
:1013700000F1604083F8001300F5614001239340C1
:10138000C0F8803103607047F8B515468268066979
:10139000AA420B46816938BF8568761AB542044671
:1013A00007D218462A46FFF737FDA3692B44A361ED
:1013B0000DE011D932461846FFF72EFDAF1B3A4615
:1013C000E1683044FFF728FDE2683A44A261A3686F
:1013D0005B1BA3602846F8BD18462A46FFF71CFD94
:1013E000E368E4E783682DE9F0410446934215463B
:1013F000266938BF85684069361AB5420F4606D25D
:101400002A46FFF709FD63692B4463610DE012D999
:101410003246A5EB0608FFF7FFFC4246B919E06823
:10142000FFF7FAFCE26842446261A3685B1BA360B9
:101430002846BDE8F0812A46FFF7EEFCE368E4E7C2
:1014400010B50A440024C361029B006040608460C0
:10145000C160816141610261036210BD08B58269AA
:101460004369934201D1826882B982680132826005
:101470005A1C42611970426903699A4201D3C368D8
:101480004361002100F09CFE002008BD4FF0FF30BA
:1014900008BD000070B5202304460E4683F3118872
:1014A000A568A5B1A368A269013BA360531CA36111
:1014B00015782269934224BFE368A361E3690BB105
:1014C00020469847002383F31188284670BD314693
:1014D000204600F065FE0028E2DA85F3118870BD31
:1014E0002DE9F74F05460F4690469A46D0F81C90D6
:1014F000202686F311884FF0000B144664B1224673
:1015000039462846FFF740FF034668B9514628464A
:1015100000F046FE0028F1D0002383F31188A8EBE9
:10152000040003B0BDE8F08FB9F1000F03D00190C3
:101530002846C847019B8BF31188E41A1F4486F3A1
:101540001188DBE7C16081614161C3611144009B87
:10155000006040608260016103627047F8B5044634
:101560000E461746202383F31188A568A5B1A3680A
:10157000013BA36063695A1C62611E702369626942
:101580009A4224BFE3686361E3690BB12046984740
:10159000002080F31188F8BD3946204600F000FE97
:1015A0000028E2DA85F31188F8BD000083694269FA
:1015B0009A4210B501D182687AB98268013282609C
:1015C0005A1C82611C7803699A4201D3C368836103
:1015D000002100F0F5FD204610BD4FF0FF3010BD9A
:1015E0002DE9F74F05460F4690469A46D0F81C90D5
:1015F000202686F311884FF0000B144664B1224672
:1016000039462846FFF7EEFE034668B9514628469C
:1016100000F0C6FD0028F1D0002383F31188A8EB69
:10162000040003B0BDE8F08FB9F1000F03D00190C2
:101630002846C847019B8BF31188E41A1F4486F3A0
:101640001188DBE7026843681143016003B1184762
:10165000704700001430FFF743BF00004FF0FF3326
:101660001430FFF73DBF00003830FFF7B9BF00006E
:101670004FF0FF333830FFF7B3BF00001430FFF7EF
:1016800009BF00004FF0FF311430FFF703BF000027
:101690003830FFF763BF00004FF0FF323830FFF7FC
:1016A0005DBF000000207047FFF774BD044B03606E
:1016B000002343608360C36001230374704700BF4D
:1016C000183D000810B52023044683F31188FFF766
:1016D000DDFD02232374002383F3118810BD000075
:1016E00038B5C36904460D461BB904210844FFF709
:1016F000A9FF294604F11400FFF7B0FE002806DA1E
:10170000201D4FF48061BDE83840FFF79BBF38BD16
:10171000026843681143016003B118477047000035
:1017200013B5446BD4F894341A681178042915D190
:10173000217C022912D11979128901238B4013428D
:101740000CD101A904F14C0001F0ACFED4F8944492
:10175000019B21790246206800F0E0F902B010BD3B
:10176000143001F02FBE00004FF0FF33143001F0B1
:1017700029BE00004C3001F001BF00004FF0FF33E4
:101780004C3001F0FBBE0000143001F0FDBD000044
:101790004FF0FF31143001F0F7BD00004C3001F084
:1017A000CDBE00004FF0FF324C3001F0C7BE00004C
:1017B000D0F8942438B5136819780429054601D067
:1017C000012038BD017C0229FAD112795C890120FF
:1017D00090400440F4D105F1140001F08FFD024661
:1017E0000028EDD0D5F894544FF4807328686979B7
:1017F00000F082F9204638BD406BFFF7D9BF0000EA
:1018000000207047704700007FB5124B0360002333
:1018100043608360C360012502260F4B05740446B4
:101820000290019300F18402294600964FF48073E0
:10183000143001F03FFD094B0193029400964FF4E0
:10184000807304F52372294604F14C0001F006FE72
:1018500004B070BD403D0008F917000821170008CA
:101860000B68202282F311880A7903EB820210624E
:101870004A790D3243F822008A7912B103EB8203D0
:10188000186202230374C0F89414002383F31188B0
:101890007047000038B5037F044613B190F8543008
:1018A000ABB9201D01250221FFF732FF04F114001E
:1018B00025776FF0010100F08FFC84F8545004F19B
:1018C0004C006FF00101BDE8384000F085BC38BD28
:1018D00010B5012104460430FFF71AFF00232377D7
:1018E00084F8543010BD000038B50446002514308B
:1018F00001F0F8FC04F14C00257701F0C7FD201D34
:1019000084F854500121FFF703FF2046BDE838401A
:10191000FFF74EBF90F85C3003F06003202B19D125
:1019200090F85D20212A0AD0222A4FF000030ED021
:10193000202A0FD1084A02650722426504E0064BBF
:101940000365072343650023836501207047036512
:101950004365F9E70020704728240220D0F894342A
:1019600037B51A681178042904461AD1017C022976
:1019700017D11979128901238B40134211D100F13B
:101980004C05284601F042FE58B101A9284601F055
:1019900089FDD4F89444019B21790246206800F027
:1019A000BDF803B030BD000000EB8103F7B51C6A41
:1019B00005460E46F4B1202383F3118805EB860714
:1019C000201D0821FFF7A4FEFB685B691B684C34EF
:1019D00013B1204601F074FD01A9204601F062FD1B
:1019E000024648B1019B3146284600F097F8002393
:1019F00083F3118803B0F0BDFB685A691268002AAE
:101A0000F5D01B8A013B1340F1D105F15C02EAE7F6
:101A10000D3138B550F82140DCB1202383F3118813
:101A2000D4F894241368527903EB8203DB689B6932
:101A30005D6845B104216018FFF76AFE294604F18C
:101A4000140001F065FC2046FFF7B2FE002383F38B
:101A5000118838BD7047000001F012B801230370EF
:101A60000023436000F1240200F1380142F8043BF6
:101A70008A421361FAD103814381704738B5044625
:101A8000202383F3118800254160C560056145610D
:101A90008561C561056201F003F80223237085F3B7
:101AA000118838BD70B500EB810305465069DA60D6
:101AB0000E46144618B110220021FFF7D7F9A0698D
:101AC00018B110220021FFF7D1F931462846BDE8B0
:101AD000704001F0AFB80000028902F001020281FB
:101AE000428902F001024281002202614261826168
:101AF000C261026201F032B9F0B400EB810447899F
:101B0000E4680125A4698D403D434581236000239D
:101B1000A2606360F0BC01F04DB90000F0B400EBCE
:101B200081040789E468012564698D403D4305818E
:101B300023600023A2606360F0BC01F0C7B900001D
:101B400070B50223002504460370A0F8645080F8A5
:101B5000665080F8675005814581C5600561456123
:101B60008561C561056280F84C5000F0FFFF636835
:101B70001B6823B129462046BDE87040184770BD58
:101B8000436802781B6880F86820052202700BB158
:101B90000421184770470000436890F868201B68CC
:101BA00002700BB1052118477047000090F84C30C7
:101BB00070B5044613B1002380F84C3004F15C0288
:101BC000204601F0EDF863689B6863BB94F85C50B5
:101BD00015F0600615D194F85D3005F07F0545EAF3
:101BE000032540F202339D4200F00E815BD8022DA6
:101BF00000F0DC803FD8002D00F08780012D00F040
:101C0000CF800021204601F037FB0021204601F063
:101C100029FB63681B6813B10621204698470623F9
:101C200084F84C3070BD204698470028CED094F8F8
:101C3000632094F8623043EA0223626D934238BF16
:101C4000636594F95C30656D002B4FF0200380F2E2
:101C5000FD80002D00F0EC80092284F84C2083F3F5
:101C600011880021636D226D2046FFF757FF002386
:101C700083F3118870BDB5F5817F00F0B180B5F5B3
:101C8000407F49D0B5F5807FBBD194F85E30012B01
:101C9000B7D1B4F8643023F00203A4F864302665A9
:101CA0006665A665C3E740F201639D421ED8B5F59F
:101CB000C06F3BD2B5F5A06FA3D1B4F85C30B3F5DB
:101CC000A06F0ED194F85E3084F86630204600F0A4
:101CD000A5FF63681B6813B10121204698470323C1
:101CE0002370002323656365A365A0E7B5F5106F36
:101CF00032D040F602439D4252D0B5F5006F80D1FC
:101D000004F167032365012324E004F164032365E0
:101D100002236365A5658AE794F85E30012B7FF4A2
:101D200070AFB4F8643043F00203B6E794F8612072
:101D3000616894F860304D6894F85F1043EA0223BC
:101D4000204694F85E20A84700283FF45AAF436825
:101D5000236503686365A4E72378042B10D120234F
:101D600083F311882046FFF7B7FE86F31188636876
:101D700084F867601B68032121700BB120469847E7
:101D800094F85E30002BACD084F8673004232370C5
:101D900063681B68002BA4D0022120469847A0E767
:101DA000374B23650223636500239DE794F8601099
:101DB00011F0800F204601F00F010ED000F0E2FF7D
:101DC000012806D002287FF41CAF2E4B23656065E6
:101DD00067E72D4B2365656563E700F0C5FFEFE717
:101DE00094F85E30002B7FF40CAF94F8603013F061
:101DF0000F013FF476AF1A06204602D501F050FAE3
:101E00006FE701F043FA6CE794F85E30002B7FF443
:101E1000F8AE94F8603013F00F013FF462AF1B0688
:101E2000204602D501F028FA5BE701F01BFA58E7DB
:101E3000142284F84C2083F311882B462A46294625
:101E40002046FFF759FE85F3118870BD5DB115225C
:101E500084F84C2083F311880021636D226D2046A5
:101E6000FFF74AFE03E70B2284F84C2083F3118826
:101E70002B462A4629462046FFF750FEE3E700BFDF
:101E8000703D0008683D00086C3D000838B590F8CA
:101E90004C300446152B29D8DFE803F03E282828CB
:101EA00028283E28280B29392828282828282828A7
:101EB0003E3E90F8631090F86220436D42EA0122A2
:101EC0009A4214D9C268128AB3FBF2F502FB1535A7
:101ED0006DB9202383F311882B462A462946FFF744
:101EE0001DFE85F311880A2384F84C3038BD142375
:101EF00084F84C30202383F3118800231A461946B6
:101F00002046FFF7F9FD002383F3118838BD836D68
:101F100003B198470023E7E7002101F0ADF9002164
:101F2000204601F09FF963681B6813B10621204623
:101F300098470623D8E7000090F84C20152A38B5BA
:101F4000044622D80123934040F6416213421DD13A
:101F500013F480150FD19B0217D50B2380F84C305A
:101F6000202383F311882B462A462946FFF7D6FD06
:101F700085F3118838BDC3689B695B682BB9836D95
:101F800003B19847002384F84C3038BD002101F09C
:101F900073F90021204601F065F963681B6813B1ED
:101FA0000621204698470623EDE70000024B002259
:101FB0001B605B609A6070478C33022000230374BF
:101FC0008268054B1B6899689142FBD25A6803608E
:101FD00042601060586070478C33022008B520239F
:101FE00083F31188037C032B05D0042B0DD02BB970
:101FF00083F3118808BD436900221A604FF0FF3354
:102000004361FFF7DBFF0023F2E790E80C001A6062
:1020100002685360F2E70000002303748268054BF6
:102020001B6899689142FBD85A680360426010604F
:10203000586070478C330220054B19690874186882
:1020400002681A605360186101230374FEF76CB9CB
:102050008C33022030B54B1C87B005460A4C10D09B
:1020600023690A4A01A800F0D3F82846FFF7E4FFE5
:10207000049B13B101A800F007F92369586907B060
:1020800030BDFFF7D9FFF8E78C330220DD1F0008D1
:1020900038B50C4D41612B6981689A6891420446BC
:1020A00003D8BDE83840FFF789BF1846FFF786FF21
:1020B00001232C61014623742046BDE83840FEF719
:1020C00033B900BF8C330220044B1A681B69906837
:1020D0009B68984294BF0020012070478C330220F7
:1020E00010B5084C236820691A68226054600122E8
:1020F00023611A74FFF790FF01462069BDE8104084
:10210000FEF712B98C330220826002220274002290
:10211000427470478368A3F17C0243F80C2C026977
:1021200043F83C2C426943F8382C074A43F81C2CEE
:10213000C26843F8102C022203F8082C002203F88E
:10214000072CA3F1180070474103000810B52023A5
:1021500083F31188FFF7DEFF00210446FFF798FFA5
:10216000002383F31188204610BD0000024B1B6939
:1021700058610F20FFF760BF8C330220202383F3C8
:102180001188FFF7F3BF000008B50146202383F351
:1021900011880820FFF75EFF002383F3118808BD34
:1021A00049B1064B42681B6918605A60136043606E
:1021B0000420FFF74FBF4FF0FF3070478C330220F1
:1021C0000368984206D01A68026050605961184648
:1021D000FFF7F4BE7047000038B504460D4620688E
:1021E000844200D138BD036823605C604561FFF71D
:1021F000E5FEF4E7054B03F114025A619A614FF0D2
:10220000FF32DA6100221A62704700BF8C3302206D
:10221000F8B503614FF08043C2605C6A194B1A46FF
:10222000022952F8145F38BF0221954206461F4624
:102230000AD1586198611C62056045608160081987
:10224000BDE8F84001F004BA186AAB68241A0C190A
:1022500002D3E41A2D6804E09C4202D2204401F02B
:1022600005FAAB689C42F4D86B68736035601E60F9
:102270006E60B460A9684FF0FF33091BA960FB6171
:10228000F8BD00BF8C33022010B41B4C234653F81A
:10229000141F814210D0416802680A6002685160D0
:1022A0009A424FF00001C16003D0936881680B44EB
:1022B00093605DF8044B70470A68626100209A429F
:1022C0005360C86003D15DF8044B01F0C9B993684D
:1022D0008868034493604FF08042206A526A121A61
:1022E0009342E6D9991A012998BF931C18445DF8C6
:1022F000044B01F0BBB900BF8C33022000207047B3
:10230000FEE70000704700004FF0FF30704700000C
:10231000022906D0032906D00129064818BF00204B
:10232000704705487047032A9ABF044800EBC20073
:1023300000207047443E0008F83D00083024022089
:1023400070B59AB001AD064608462946144600F01D
:1023500095F82846FEF782FDC0B2431C5B0086E874
:102360001800237003236370002302341946DAB285
:10237000904204F1020401D81AB070BDEA5C04F87E
:10238000022C04F8011C0133F1E7000008B52023FA
:1023900083F311880348FFF7E1FA002383F31188E0
:1023A00008BD00BFCC33022010B50446052916D85D
:1023B000DFE801F016150316161D202383F311889C
:1023C0000E4A0121FFF76EFB20460D4A0221FFF75E
:1023D00069FB0C48FFF788FA002383F3118810BDCE
:1023E000202383F311880748FFF754FAF4E72023EA
:1023F00083F311880348FFF76BFAEDE7743D00089B
:10240000983D0008CC33022038B50C4D0C4C0D49DA
:102410002A4604F10800FFF793FF05F1CA0204F110
:1024200010000949FFF78CFF05F5CA7204F1180086
:102430000649BDE83840FFF783BF00BF943802204B
:1024400030240220C43D0008D13D0008DF3D0008D3
:1024500070B5044608460D46FEF700FDC6B220469C
:10246000013403780BB9184670BD32462946FEF791
:10247000DDFC0028F3D1012070BD00002DE9F84FEC
:1024800005460C46FEF7EAFC2B49C6B22846FFF784
:10249000DFFF08B10336F6B228492846FFF7D8FF18
:1024A00008B11036F6B2632E0DD8DFF88C80DFF855
:1024B0008C90234FDFF890A0DFF890B02E7846B9CB
:1024C0002670BDE8F88F29462046BDE8F84F01F098
:1024D000E9BB252E2CD1072241462846FEF7A6FC53
:1024E00058B9DBF800302360DBF804306360BBF8D8
:1024F0000830238107350A34E0E708224946284698
:10250000FEF794FCA0B90F4BA21C13F8011F090998
:102510005345C95D02F8021C197801F00F0102F160
:102520000202C95D02F8031CEFD118340835C5E773
:10253000267001350134C1E7643E0008DF3D000824
:10254000773E00081FF4F01F2BF4F01F6C3E0008CC
:10255000BFF34F8F024AD368DB03FCD4704700BF40
:10256000003C024008B5074B1B7853B9FFF7F0FF5A
:10257000054B1A69002ABFBF044A5A6002F188322B
:102580005A6008BDF23A0220003C02402301674530
:1025900008B5054B1B7833B9FFF7DAFF034A136917
:1025A00043F00043136108BDF23A0220003C0240B0
:1025B0000B2870B513D80B4A0B4C137863B90B4E2C
:1025C0004FF0006144F8231056F8235001330C2BD0
:1025D0002944F7D10123137054F8200070BD002066
:1025E00070BD00BF243B0220F43A0220883E000860
:1025F000014B53F820007047883E00080C207047BC
:102600000B2810B5044601D9002010BDFFF7D0FFFC
:10261000064B53F824301844C21A0BB9012010BDE0
:1026200012680132F0D1043BF6E700BF883E000893
:102630000B2810B5044621D8FFF78AFFFFF792FF59
:102640000F4AF323D360C300DBB243F4007343F0BB
:1026500002031361136943F480331361FFF778FFBA
:10266000FFF7A6FF074B53F8241000F0DDF8FFF743
:102670008FFF2046BDE81040FFF7C2BF002010BD0D
:10268000003C0240883E00082DE9F84312F00103A7
:10269000154640D18218B2F1026F3CD22C4B1B6818
:1026A00013F0010337D02B4CFFF75CFFF323E360FB
:1026B000FFF74EFF40F20127032D01D9830713D006
:1026C000244C0F46401A40F20118EB1B0B44012B1F
:1026D00000EB0706236924D823F001032361FFF7E9
:1026E00057FF0120BDE8F883236923F44073236179
:1026F00023693B43236151F8046B0660BFF34F8F9E
:10270000FFF726FF03689E4208D0236923F00103E8
:102710002361FFF73DFF0020BDE8F883043D04304E
:10272000CAE723F440732361236943EA0803236162
:10273000B94637F8023B3380BFF34F8FFFF708FFEE
:102740003688B9F80030B6B2B342BED0DDE700BF7C
:1027500000380240003C0240084908B50B7828B117
:1027600053B9FFF7FFFE01230B7008BD23B1BDE88D
:1027700008400870FFF70CBF08BD00BFF23A022006
:1027800010B50244064B0439D2B2904200D110BDBC
:10279000441C00B253F8200041F8040FE0B2F4E703
:1027A00050280040104B30B51C6F240407D41C6F18
:1027B00044F400741C671C6F44F400441C670B4C09
:1027C000236843F4807323600244094B0439D2B276
:1027D000904200D130BD441C00B251F8045F43F870
:1027E0002050E0B2F4E700BF003802400070004023
:1027F0005028004007B5012201A90020FFF7C0FFC3
:10280000019803B05DF804FB13B50446FFF7F2FF2F
:10281000A04206D002A9012241F8044D0020FFF792
:10282000C1FF02B010BD00000144BFF34F8F064B43
:10283000884204D3BFF34F8FBFF36F8F7047C3F845
:102840005C022030F4E700BF00ED00E0034B1B68A2
:102850009B0042BF024B01221A707047743802403D
:10286000253B0220014B1878704700BF253B022012
:10287000064A536823F001035360EFF3098368337A
:1028800083F30988002383F31188704730EF00E059
:1028900010B5202383F31188104B5B6813F4006399
:1028A00018D0F1EE103AEFF309844FF0807344F83A
:1028B0004C3C0B4BDB6844F8083CA4F1680383F301
:1028C0000988FFF701FC18B1064B44F8503C10BDD5
:1028D000054BFAE783F3118810BD00BF00ED00E05F
:1028E00030EF00E05103000854030008F0B5BFF3D7
:1028F0004F8FBFF36F8F1D4B0021C3F85012BFF3F2
:102900004F8FBFF36F8F5A6942F400325A61BFF3A1
:102910004F8FBFF36F8FC3F88410BFF34F8FD3F87F
:102920008020C2F3C904C2F34E325201A50743F618
:10293000E07602EA060E284621464EEA00070139F3
:10294000C3F860724F1C00F14040F6D1203A12F1FA
:10295000200FEED1BFF34F8F5A6942F480325A6193
:10296000BFF34F8FBFF36F8FF0BD00BF00ED00E0EE
:10297000FEE70000084A094B09498B4204D3094A83
:102980000021934205D3704752F8040F43F8040B1B
:10299000F3E743F8041BF4E794400008B03D02203D
:1029A000B03D0220B03D0220036F30B500229D688B
:1029B000C46E11464FF0FF3004EB421301329542D2
:1029C000C3F80019C3F81019C3F80809C3F8001BAD
:1029D000C3F8101BC3F8080BEED24FF00113C4F874
:1029E0001C3830BD890141F02001016103699B065B
:1029F000FCD4122000F0C8BE204B03EB80022DE96E
:102A0000F047D2F80CE0DD6EDEF81420461CD2F858
:102A100000C005EB063605EB4018516861450BD345
:102A2000D5F83428012303FA00F022EA0000C5F8A3
:102A300034081846BDE8F087BEF81040ACEB01033F
:102A4000A34228BF2346D8F81849A4B2B3EB840F99
:102A500010D894681F46A4F1040959F804AFC6F8C9
:102A600000A0042F01D9043FF7E71C440B449460F5
:102A70005360D2E70020BDE8F08700BF283B02206A
:102A800010B5054C2046FEF7E9FF4FF0A043E36682
:102A9000024B236710BD00BF283B0220DC3E00082C
:102AA0000378012B70B5054650D12A4BC46E98426D
:102AB0001BD1294B5A6B42F080025A635A6D42F087
:102AC00080025A655A6D5A6942F080025A615A6909
:102AD00022F080025A610E2143205B69FEF73EFC22
:102AE0001E4BE3601E4BC4F800380023C4F8003EC0
:102AF000C0232360EE6E4FF40413A3633369002BED
:102B0000FCDA012333610C2000F03EFE3369DB0761
:102B1000FCD4122000F038FE3369002BFCDA0026CA
:102B2000A6602846FFF740FF6B68C4F81068DB68B2
:102B3000C4F81468C4F81C684BB90A4BA3614FF081
:102B4000FF336361A36843F00103A36070BD064BCC
:102B5000F4E700BF283B0220003802404014004048
:102B600003002002003C30C0083C30C0F8B5C46E01
:102B7000054600212046FFF735FF296F00234FF05F
:102B800001128F68C4F834384FF00066C4F81C286E
:102B90004FF0FF3004EB431201339F42C2F800694B
:102BA000C2F8006BC2F80809C2F8080BF2D20B6831
:102BB000EA6E6B67636210231361166916F01006E4
:102BC000FBD1122000F0E0FDD4F8003823F4FE63BE
:102BD000C4F80038A36943F4402343F01003A36111
:102BE0000923C4F81038C4F814380A4BEB604FF0CE
:102BF000C043C4F8103B084BC4F8003BC4F810694C
:102C0000C4F800396B6F03F1100243F480136A6754
:102C1000A362F8BDB83E000840800010C26E90F874
:102C20006610D2F8003823F4FE6343EA0113C2F8B9
:102C3000003870472DE9F0410EB200EB86080D46D2
:102C4000D8F80C100F6807F00303022B50D0032BA9
:102C500050D03D4A3D4F012B18BF1746C46E4FEA76
:102C6000451E04EB0E030022C3F8102B8A6905F100
:102C7000100C002A40D04A8A05F158035B013A4300
:102C8000E2500123D4F81C2803FA0CF31343A644A2
:102C90004A69C4F81C380023CEF8103905F13F0307
:102CA000002A39D00A8A898B9208012988BF4A43B1
:102CB000416F04EB8303561841EA024246672946F6
:102CC0005A602046FFF78EFED8F80C301B8A43EA84
:102CD00085531F4305F148035B01E7500123D4F8F6
:102CE0001C2803FA05F51543C4F81C58BDE8F0810B
:102CF000174FB3E7174FB1E704EB4613D3F8002B98
:102D000022F40042C3F8002BD4F81C28012303FA54
:102D10000CF322EA0303BAE704EB83030E4A5A607A
:102D200004EB461629462046FFF75CFED6F800392C
:102D300023F40043C6F80039D4F81C38012202FA03
:102D400005F523EA0505CFE7008000100080041098
:102D50000080081000800C1000040002026F12684E
:102D60004267FFF721BE00005831C36E49015B582E
:102D700013F4004004D013F4001F14BF01200220FC
:102D8000704700004831C36E49015B5813F400409E
:102D900004D013F4001F14BF01200220704700006C
:102DA00000EB8101CB68196A0B6813604B685360B4
:102DB0007047000000EB810330B5DD68AA69136835
:102DC000D36019B9402B84BF402313606B8A146809
:102DD000C26E1C44013CB4FBF3F46343033323F0A1
:102DE000030302EB411043EAC44343F0C043C0F87D
:102DF000103B2B6803F00303012B09B20ED1D2F86C
:102E0000083802EB411013F4807FD0F8003B14BF68
:102E100043F0805343F00053C0F8003B02EB4112F3
:102E2000D2F8003B43F00443C2F8003B30BD000041
:102E30002DE9F041244DEE6E06EB40130446D3F825
:102E4000087BC3F8087B38070AD5D6F81438190769
:102E500006D505EB84032146DB6828465B68984766
:102E6000FA072FD5D6F81438DB072BD505EB8403EA
:102E7000D968CCB98B69488A5E68B6FBF0F200FB72
:102E800012628AB91868DA6890420DD2121A83E881
:102E90001400202383F311880B482146FFF78AFF93
:102EA00084F31188BDE8F081012303FA04F26B89F1
:102EB00023EA02036B81CB6823B121460248BDE8B7
:102EC000F0411847BDE8F081283B022000EB810368
:102ED00070B5DD68C36E6C692668E6604A0156BB52
:102EE0001A444FF40020C2F810092A6802F00302C5
:102EF000012A0AB20ED1D3F8080803EB421410F4E9
:102F0000807FD4F8000914BF40F0805040F000509A
:102F1000C4F8000903EB4212D2F8000940F0044063
:102F2000C2F80009D3F83408012202FA01F1014382
:102F3000C3F8341870BD19B9402E84BF40202060FA
:102F400020682E8A841940F00050013C1A44B4FBDA
:102F5000F6F440EAC440C6E7F8B504461E48C56E1C
:102F600005EB4413D3F80869C3F80869F10717D5CE
:102F7000D5F81038DA0713D500EB8403D9684B690C
:102F80001F68DA68974218D2D21B00271A605F6068
:102F9000202383F311882146FFF798FF87F31188D8
:102FA000330617D5D5F834280123A340134211D096
:102FB0002046BDE8F840FFF71FBD012303FA04F2E5
:102FC000038923EA020303818B68002BE8D02146A2
:102FD0009847E5E7F8BD00BF283B0220A0482DE94F
:102FE000F84FC56E6E69AB691E4016F4805F6E6166
:102FF000044605D0FEF7A4FDBDE8F84FFFF748BC36
:10300000002E12DAD5F8003E95489B071EBFD5F872
:10301000003E23F00303C5F8003ED5F8043823F042
:103020000103C5F80438FEF7B7FD370502D58C4813
:10303000FEF7A6FDB0040CD5D5F8083813F0060F3E
:10304000EB6823F470530CBF43F4105343F4A053C4
:10305000EB60310704D56368DB680BB180489847A3
:10306000F2026FD4B3020CD5D4F86C80DFF8F0A173
:1030700000274FF00109236F9B68F9B28B4280F063
:103080009C80F70619D5E16E0A6AC2F30A1702F0AE
:103090000F0302F4F012B2F5802F00F0B680B2F503
:1030A000402F0AD104EB830301F58051DB68186AD5
:1030B00000231A469F4240F09C803303D5F81848FD
:1030C0001DD5E70302D50020FFF7B2FEA50302D508
:1030D0000120FFF7ADFE600302D50220FFF7A8FE36
:1030E000210302D50320FFF7A3FEE20202D504204C
:1030F000FFF79EFEA30202D50520FFF799FE770396
:103100007FF57AAFE60702D50020FFF725FFA50778
:1031100002D50120FFF720FF600702D50220FFF74C
:103120001BFF210702D50320FFF716FFE20602D599
:103130000420FFF711FFA3067FF55EAF0520FFF720
:103140000BFF59E7D4F86C80DFF814A100274FF08B
:103150000109236F9B685FFA87FB5B4582D308EB0D
:103160004B13D3F8002902F44022B2F5802F22D16C
:10317000D3F80029002A1EDAD3F8002942F0904241
:10318000C3F80029D3F80029002AFBDB5946E06E7A
:10319000FFF728FC228909FA0BF322EA03032381B3
:1031A00004EB8B03DB689B6813B159465046984784
:1031B0005846FFF721FC0137CBE708EB4112D2F864
:1031C000003B03F44023B3F5802F10D1D2F8003B2D
:1031D000002B0CDA628909FA01F322EA0303638106
:1031E00004EB8103DB68DB680BB15046984701377D
:1031F00041E79C0708BF0A68072B98BF027003F1DC
:1032000001039CBF120A013054E7023304EB83022E
:1032100001F58051526890690268D0F808C0406892
:10322000A2EB000E0022104697420AD104EB830461
:1032300063689B699A683A449A605A6817445F6069
:103240003BE712F0030F08BF0868964588BF8CF86B
:10325000000002F1010284BF000A0CF1010CE3E757
:10326000283B0220C36E03EB4111D1F8003B43F42D
:103270000013C1F8003B7047C36E03EB4111D1F856
:10328000003943F40013C1F800397047C36E03EBF3
:103290004111D1F8003B23F40013C1F8003B704703
:1032A000C36E03EB4111D1F8003923F40013C1F8C8
:1032B0000039704730B5039C0172043304FB0325C9
:1032C000C361049B03630021059B00604060C160F3
:1032D000426102618561046242628162C16243634C
:1032E00030BD00000022416A41610161C26082621A
:1032F000C2626FF00101FEF76FBF0000036942690F
:10330000934203D1C2680AB100207047181D70476C
:1033100003691960C2680132C260C26913448269DC
:103320000361934224BF436A03610021FEF748BF53
:1033300038B504460D46E3683BB16269131D126857
:10334000A3621344E362002038BD237A33B92946CF
:103350002046FEF725FF0028EDDA38BD6FF00100AA
:10336000FBE70000C368C269013BC36043691344C3
:1033700082694361934224BF436A436100238362AD
:10338000036B03B11847704770B52023044683F3DD
:103390001188866A3EB9FFF7CBFF054618B186F360
:1033A0001188284670BDA36AE26A13F8015BA36224
:1033B000934202D32046FFF7D5FF002383F3118801
:1033C000EFE700002DE9F84F04460E469046994677
:1033D000202787F311880025AA46D4F828B0BBF12E
:1033E000000F09D149462046FFF7A2FF20B18BF319
:1033F00011882846BDE8F88FA16AE36AA8EB050B9F
:103400005B1A9B4528BF9B46BBF1400F1BD9334637
:1034100001F1400251F8040B43F8040B9142F9D139
:10342000A36A40334036A3624035A26AE36A9A42F7
:1034300002D32046FFF796FF8AF311884545D8D27C
:1034400087F31188C9E730465A46FDF7E5FCA36AC1
:103450005B445E44A3625D44E7E7000010B5029C54
:103460000172043303FB0421C36100238362C3623E
:10347000039B0363049B00604060C460426102617F
:10348000816104624262436310BD0000026AC2604F
:10349000426A4261026100228262C2626FF00101EF
:1034A000FEF79ABE436902699A4203D1C2680AB123
:1034B00000207047184650F8043B0B60704700002E
:1034C000C368C2690133C3604369134482694361BD
:1034D000934224BF436A43610021FEF771BE00009E
:1034E00038B504460D46E3683BB123691A1DA26254
:1034F000E2691344E362002038BD237A33B92946D8
:103500002046FEF74DFE0028EDDA38BD6FF00100D1
:10351000FBE7000003691960C268013AC260C26932
:10352000134482690361934224BF436A0361002309
:103530008362036B03B118477047000070B5202306
:1035400004460E4683F31188856A35B91146FFF7A4
:10355000C7FF10B185F3118870BDA36A1E70A36AFE
:10356000E26A01339342A36204D3E169204604393D
:10357000FFF7D0FF002080F3118870BD2DE9F84FD0
:1035800004460D4691469A464FF0200888F311886C
:103590000026B346A76A4FB951462046FFF7A0FF61
:1035A00020B187F311883046BDE8F88FA06AE76A3A
:1035B000A9EB06033F1A9F4228BF1F46402F1BD985
:1035C00005F1400355F8042B40F8042B9D42F9D136
:1035D000A36A4033A3624036A26AE36A9A4204D3E4
:1035E000E16920460439FFF795FF8BF311884E45BA
:1035F000D9D288F31188CDE729463A46FDF70CFC6D
:10360000A36A3B443D44A3623E44E5E70269436943
:103610009A4203D1C3681BB9184670470023FBE7E1
:10362000836A002BF8D0043B9B1AF5D01360C36863
:10363000013BC360C3691A44836902619A4224BF93
:10364000436A0361002383620123E5E700F042B986
:103650004FF08043002258631A610222DA607047FB
:103660004FF080430022DA60704700004FF0804343
:1036700058637047FEE7000010B5194CFEF796FC42
:10368000FEF7B8FD802217492046FEF73DFD0123D5
:1036900044F8180C0374144B144AD96821F4E061FF
:1036A0000904090C0A431249DA60CA6842F08072C0
:1036B000CA60104A1049C2F8B01F116841F00101F8
:1036C00011601022DA77202283F82220002383F36E
:1036D000118862B60948BDE81040FEF737BD00BF4B
:1036E000B4330220E83E000800ED00E00003FA05D4
:1036F000F0ED00E0001000E055CEACC5F03E000853
:103700002DE9F84F1F4C4FF00008656904F11407CC
:10371000C1464FF08043266A5B6AAA689E1B9642A8
:103720001DD34FF0200AAA68236AD5F80CB01344C1
:1037300023622B68BB425F60A6EB02066361C5F89B
:103740000C8001D1FFF78CFF89F311882869D847D5
:103750008AF311886569AB689E42E4D2D9E7626951
:10376000BA420CD0916823628E1B9660A86802282A
:103770002CBF1818981CBDE8F84FFFF777BFBDE8BD
:10378000F88F00BF8C330220034B59685A68521AD5
:103790009042FBD8704700BF001000E04B684360C8
:1037A0008B688360CB68C3600B6943614B690362BC
:1037B0008B6943620B6803607047000008B5274BB4
:1037C00027481A6940F2FF710A431A611A6922F404
:1037D000FF6222F007021A611A691A6B0A431A6320
:1037E0001A6D0A431A651F4A1B6D1146FFF7D6FF73
:1037F0001D4802F11C01FFF7D1FF1C4802F13801FE
:10380000FFF7CCFF1A4802F15401FFF7C7FF194830
:1038100002F17001FFF7C2FF174802F18C01FFF7B8
:10382000BDFF164802F1A801FFF7B8FF144802F1E6
:10383000C401FFF7B3FF134802F1E001FFF7AEFF49
:10384000114802F1FC01FFF7A9FF104802F58C7145
:10385000FFF7A4FFBDE8084000F09EB80038024022
:1038600000000240103F000800040240000802402F
:10387000000C0240001002400014024000180240F8
:10388000001C0240002002400024024000280240A8
:1038900008B500F0F5F9FFF7EFFEFEF7D7FFBDE83A
:1038A0000840FEF7B1BD0000704700004FF08043B4
:1038B00010B51A69920708D500241C61202383F3F0
:1038C0001188FFF71DFF84F31188BDE81040FEF753
:1038D000DFBF0000104B1A6C42F001021A641A6E2E
:1038E00042F001021A660D4A1B6E936843F0010311
:1038F00093604FF080436B229A624FF0FF32DA629E
:1039000000229A615A63DA605A6001225A610821E2
:103910001A601C20FDF722BD00380240002004E0A0
:103920001B4B1A696FEA42526FEA52521A611A69C6
:10393000C2F30A021A614FF0FF301A695A695861DE
:1039400000215A6959615A691A6A62F080521A62F2
:103950001A6A02F080521A621A6A5A6A58625A6ADD
:1039600059625A6A0B4A106840F480701060186FF0
:1039700000F44070B0F5007F1EBF4FF48030186730
:103980001967536823F40073536000F059B900BFFE
:103990000038024000700040354B364A1A64364AFF
:1039A0004FF4404111601A6842F001021A601A682F
:1039B0009207FCD59A6822F003029A602C4B1946B4
:1039C0009A6812F00C02FBD1186800F0F900186038
:1039D0009A601A6842F480321A600B689B03FCD527
:1039E0004B6F43F001034B67214B5A6F9007FCD597
:1039F000224A5A601A6842F080721A601E4B1A46B8
:103A000059684904FCD5196841F48031196053683C
:103A1000D803FCD5136843F400331360164A536887
:103A20009903FCD5124B1A689201FCD5144A9A608E
:103A300040F20112C3F88C200022C3F89020114AF2
:103A400040F2073111609A6842F002029A60084B16
:103A50009A6802F00C02082AFAD15A6C42F48042A9
:103A60005A645A6E42F480425A665B6E704700BFD9
:103A7000003802400004001000700040186C40093B
:103A800000948838003C0240084A08B55369116820
:103A90000B4003F00103536123B1054A13680BB1D6
:103AA00050689847BDE80840FEF7F2BE003C014070
:103AB000C8250220084A08B5536911680B4003F075
:103AC0000203536123B1054A93680BB1D06898474C
:103AD000BDE80840FEF7DCBE003C0140C8250220DE
:103AE000084A08B5536911680B4003F00403536199
:103AF00023B1054A13690BB150699847BDE80840E6
:103B0000FEF7C6BE003C0140C8250220084A08B5A1
:103B1000536911680B4003F00803536123B1054A50
:103B200093690BB1D0699847BDE80840FEF7B0BE75
:103B3000003C0140C8250220084A08B553691168B5
:103B40000B4003F01003536123B1054A136A0BB114
:103B5000506A9847BDE80840FEF79ABE003C014015
:103B6000C8250220174B10B55C691A68144004F48C
:103B700078725A61A30604D5134A936A0BB1D06ACE
:103B80009847600604D5104A136B0BB1506B9847E9
:103B9000210604D50C4A936B0BB1D06B9847E20514
:103BA00004D5094A136C0BB1506C9847A30504D592
:103BB000054A936C0BB1D06C9847BDE81040FEF7F6
:103BC00067BE00BF003C0140C82502201A4B10B55B
:103BD0005C691A68144004F47C425A61620504D599
:103BE000164A136D0BB1506D9847230504D5134A3F
:103BF000936D0BB1D06D9847E00404D50F4A136E56
:103C00000BB1506E9847A10404D50C4A936E0BB1CA
:103C1000D06E9847620404D5084A136F0BB1506FF9
:103C20009847230404D5054A936F0BB1D06F98478A
:103C3000BDE81040FEF72CBE003C0140C825022024
:103C4000062108B50846FDF789FB06210720FDF788
:103C500085FB06210820FDF781FB06210920FDF7E1
:103C60007DFB06210A20FDF779FB06211720FDF7D1
:103C700075FB06212820BDE80840FDF76FBB00005A
:103C800008B5FFF74DFEFDF7B5F9FDF70DFDFDF7A2
:103C9000E3FEFDF7B7FDFFF707FEBDE80840FFF7BD
:103CA000D5BC0000034611F8012B03F8012B002AB4
:103CB000F9D17047121012131211000000104100C8
:103CC00001105A00CC33022048260220B4260220DC
:103CD0002027022053544D3332463F3F3F3F3F3F62
:103CE0000053544D333246375B347C355D78005396
:103CF000544D333246375B367C375D780000000028
:103D0000009600000000000000000000000000001D
:103D10000000000000000000000000007116000814
:103D20005D1600089916000885160008911600080F
:103D30007D1600086916000855160008A51600082B
:103D4000000000007D17000869170008A51700088B
:103D5000911700089D1700088917000875170008BB
:103D600061170008011800080000000001000000B1
:103D7000000000000200000000000000A919000877
:103D8000111A0008400040006438022074380220F4
:103D9000020000000000000003000000000000001E
:103DA000551A0008000000001000000084380220AE
:103DB000000000000100000000000000283B02207D
:103DC000010102004865782F50726F6669434E43C7
:103DD000004375626559656C6C6F772D424C002508
:103DE00053455249414C2500A923000811230008DE
:103DF000151900088D23000843000000003E00084C
:103E000009024300020100C032090400000102025D
:103E10000100052400100105240100010424020210
:103E20000524060001070582030800FF09040100BC
:103E3000020A000000070501024000000705810298
:103E400040000000120000004C3E0008120110016A
:103E500002000040AE2D021000020102030100002A
:103E60000403090425424F4152442500437562650D
:103E700059656C6C6F7700303132333435363738F2
:103E80003941424344454600008000000080000064
:103E9000008000000080000000000200000004001C
:103EA0000000040000000400000004000000040002
:103EB000000004000000040000000000AD1B00082A
:103EC0008D1E0008391F000840004000A03B022062
:103ED000A03B022001000000B03B02208000000057
:103EE00040010000050000006D61696E00000000E7
:103EF000083F0008B83B0220B03D0220010000004E
:103F0000753600080000000069646C650000000060
:103F10000000802A00000000AAAAAAAA000000004F
:103F2000FFFF00000000000000A00A0000010000E8
:103F300000000000AAAAAAAA00000000FFFF0000DB
:103F40000000000000000000000000000000000071
:103F5000AAAAAAAA00000000FFFF000000000000BB
:103F60000000000080298A0100000000AAAAAAAA75
:103F700040154501FFFF00000070700777700000DA
:103F80000080020000000000AAAAAAAA00400100C6
:103F9000FFFF00000000008008000000000000009B
:103FA00000000000AAAAAAAA00000000FFFF00006B
:103FB0000000000000000000000000000000000001
:103FC000AAAAAAAA00000000FFFF0000000000004B
:103FD000000000000000000000000000AAAAAAAA39
:103FE00000000000FFFF00000000000000000000D3
:103FF0000000000000000000AAAAAAAA0000000019
:10400000FFFF0000000000000000000000000000B2
:1040100000000000000000000000000000000000A0
:104020000000000000000000000000000000000090
:104030000000000000000000000000000000000080
:104040000000000000000000FF0000000000000071
:10405000D43C00083F00000049040000E13C000897
:104060003F00000051040000EF3C00083F0000004A
:10407000009600000000080004000000603E0008F8
:104080000000000000000000000000000000000030
:08409000000000000000000028
:00000001FF
